:020000040000FA
:1000000030050020D5000000C90A00003D0A0000AC
:1000100000000000000000000000000000000000E0
:10002000000000000000000000000000390B00008C
:1000300000000000000000000D0B00003D0B000060
:10004000E7000000E7000000E7000000E700000014
:10005000E7000000E7000000E7000000E700000004
:10006000E7000000E7000000E7000000E7000000F4
:10007000E70000000000000000000000E7000000B2
:10008000E700000000000000E7000000E7000000BB
:1000900000000000E700000000000000ED0C000080
:1000A000E7000000E7000000000000000000000082
:1000B000E7000000E700000000000000E70000008B
:1000C0000348854600F012F9004800474513000038
:1000D000300500200448804704480047FEE7FEE75B
:1000E000FEE7FEE7FEE7FEE7790B0000C100000037
:1000F00030B50B46014600202022012409E00D46C0
:10010000D5409D4205D31D469540491B2546954047
:1001100040191546521E002DF1DC30BDD2B201E06F
:100120000270401C491EFBD270470022F6E710B552
:1001300013460A4604461946FFF7F0FF204610BD55
:1001400070B502464A40D50F40004A00ED0740080E
:100150005208002814D0002A12D0C40DD30D410239
:100160000120C0055202490A520AE41A091812185D
:100170007D34914201D3641C00E04900002C01DA77
:10018000002070BD0023914201D3891A0343400827
:1001900049000028F7D100290AD0914202D101215B
:1001A000C90705E0914201D2012101E00121C943C3
:1001B000E005C018401900F058F870BD420005D0A5
:1001C0004200120E52428A4201DB00207047C905EC
:1001D0000818704710B500229623114600F04DF81C
:1001E00010BD410040020122400AD205090E8018CC
:1001F0007F2901DA00207047962903DC9622511AE4
:10020000C8407047963988407047C20FD2074000F7
:1002100040080BD0C10D0723DB01C91840020905B6
:10022000400A1143C20840071143704700200146AD
:100230007047CB0FDB07490010B5490802460A4357
:1002400007D00A0D07240903E401090B121B002A39
:1002500001DC002010BDC900440F0C43C100E018B0
:10026000D205801800F001F810BD002904DA401C06
:10027000490001D140084000704770B40024050CCB
:1002800005D11024000402D1002921D01124050E2B
:1002900001D100020834050F01D10001241D850F92
:1002A00001D18000A41C002801DB4000641C00294F
:1002B00008D020252E1B0D46F540A14000D001217D
:1002C0002943084301061B1B000ADB1D02D5002041
:1002D00070BC7047DB05181880180029F8DA401C3C
:1002E0004900F5D170BC400840007047064C01251C
:1002F000064E05E0E36807CC2B430C3C98471034CE
:10030000B442F7D3FFF7E0FEA41B0000C41B0000BB
:1003100030B585B0012568460573457300248473A4
:1003200003A9102000F035F96846047002214170DD
:100330008470C47005710821417184710A210172B1
:100340000321C17100F014F805B030BD03484068C6
:10035000800701D500207047012070470010004041
:10036000024800680005000D7047000000100040C2
:1003700030B503460078012817D85878072814D8D4
:100380009878012811D8D87803280ED8187902282F
:100390000BD85879132808D89879012805D8187AE5
:1003A0001F2802D8D879032801D9002030BD00F0D9
:1003B00059F82B4908680124204308600868042282
:1003C000104308602648403882680514AA438260BA
:1003D000C2685D7952095201ED06ED0E2A43C260F2
:1003E00082680825AA431D78ED072D0F2A438260F5
:1003F00082685D78D208D2006D076D0F2A43826053
:10040000826803252D02AA43DD78AD07AD0D2A438E
:100410008260826805152A4382600A680225AA4321
:100420000A608168821491439A79D207D20C1143F1
:10043000816081681F22120491431A7AD206D20A7F
:1004400011438160416830229143DA799207920E1C
:1004500011434160416821434160012030BD0000EB
:100460004010004008480021416041221203826090
:100470008215C260016141618162044A02630248DF
:100480004030016070470000001000400000FF0F86
:1004900006488168C90401D500207047816801229F
:1004A000520311438160012070470000001000409A
:1004B00006488168C90401D500207047816801227F
:1004C00052039143816001207047000000100040FA
:1004D000012189070868C007C00F01D0054A0A60DA
:1004E0000022054BD2439A60002801D0002008600A
:1004F000704700009669AA554000004000B503000F
:1005000000F0BAFC2B171945454545454527292BD1
:100510002D2F3145191B1D1F21232527292B2D2F59
:10052000313335374545454545393B3D3F454143E9
:100530004500002000BD012000BD022000BD0320B9
:1005400000BD042000BD052000BD062000BD072021
:1005500000BD082000BD092000BD0A2000BD0B2001
:1005600000BD0C2000BD0D2000BD0E2000BD0F20E1
:1005700000BD102000BD162000BD172000BD1820B2
:1005800000BD192000BD1B2000BD1C2000BDFF20A8
:1005900000BD30B5054608780C4601280FD0002173
:1005A000284600F0DBF9A178284600F073F861785E
:1005B000284600F059F86078002812D019E001218F
:1005C000284600F0CBF90121284600F04DF8002123
:1005D000284600F05FF80021284600F077F9002156
:1005E00010E02179284600F027F8E178284600F04D
:1005F0003DF90121284600F099F96179284600F07B
:1006000065F9A179284600F049F90021284600F053
:1006100075F930BD00B50146FFF770FF0D2901D80F
:10062000044901E0034980390968C140C807C00F87
:1006300000BD00008004004010B50446FFF75EFFD7
:1006400001220D2C03D8074B03E0596010BD054B68
:10065000803B0029596802D082401143F5E782406F
:100660009143F2E7C004004010B50446FFF746FF8F
:1006700001220D2C07D8064B07E082409A6110BD7D
:100680008240DA6110BD024B803B0129F8D1F4E7CA
:1006900080040040F0B5002906D0012904D00229C9
:1006A00002D0032900D0FF2130256F4A6E4C2E0264
:1006B0002F03803A030000F0DFFB2B171D232323B9
:1006C000232323242A2F363B4023494E555A5F6665
:1006D0006D767C81888D9299A0A92323232323AF53
:1006E000B6BFC523CACF2300606A8907800880008F
:1006F000890F03E0606A8907A843890E0843606296
:10070000F0BDA06A890780088000890F1BE0A06AFD
:100710008907A843890E16E0A06A032212029043BB
:100720008907890D0FE0A06A8907B043890C0AE0A8
:10073000A06A8907B843890B05E0A06A0322120565
:1007400090438907890A0843A062F0BD506A89076F
:10075000A843890E24E0506A03231B0298438907AB
:10076000890D1DE0506A8907B043890C18E0506A72
:100770008907B843890B13E0506A03231B0598438C
:100780008907890A0CE0506A03231B0698438907EE
:10079000890905E0506A03231B07984389078908E4
:1007A00008435062F0BD906A890780088000890F75
:1007B00029E0906A8907A843890E24E0906A032300
:1007C0001B0298438907890D1DE0906A8907B04391
:1007D000890C18E0906A8907B843890B13E0906A86
:1007E00003231B0598438907890A0CE0906A0323B9
:1007F0001B0698438907890905E0906A03231B07B4
:1008000098438907890808439062F0BDD06A890738
:1008100080088000890F0CE0D06A03231B069843F0
:100820008907890905E0D06A03231B0798438907D4
:1008300089080843D062F0BD106B890780088000EA
:10084000890F0DE0106B8907A843890E08E0106B33
:100850008907B043890C03E0106B8907B843890B03
:1008600008431063F0BD00008004004010B504464A
:10087000FFF744FE01220D2C03D8074B03E09963D8
:1008800010BD054B803B0029996B02D0824011437B
:10089000F5E782409143F2E78004004010B504463A
:1008A000FFF72CFE01220D2C03D8074B03E0196043
:1008B00010BD054B803B0029196802D082401143CE
:1008C000F5E782409143F2E7C004004010B50446CA
:1008D000FFF714FE01220D2C03D8074B03E0D96368
:1008E00010BD054B803B0029D96B02D082401143DB
:1008F000F5E782409143F2E78004004010B50446DA
:10090000FFF7FCFD01220D2C03D8074B03E0D96053
:1009100010BD054B803B0029D96802D082401143AD
:10092000F5E782409143F2E7C004004010B5044669
:10093000FFF7E4FD01220D2C03D8074B03E099607B
:1009400010BD054B803B0029996802D082401143BD
:10095000F5E782409143F2E7C004004010B5044639
:10096000FFF7CCFD01220D2C03D8074B03E05963A0
:1009700010BD054B803B0029596B02D082401143CA
:10098000F5E782409143F2E78004004010B5044649
:10099000FFF7B4FD01220D2C07D8064B07E082407B
:1009A0009A6010BD8240DA6010BD024B803B012985
:1009B000F8D1F4E78004004030B501241D4BA407B2
:1009C000236002251C4B012858680DD040084000C8
:1009D00058605868A8435860186880088000401C18
:1009E00018600020206030BD800309D4586840089A
:1009F0004000586058682843586058688003FCD508
:100A0000206A00090001401C206258680C258907F3
:100A1000A843090F08435860012A03D0586880038F
:100A2000FCD5DEE7186880088000186058688003ED
:100A3000FCD5D6E79669AA5540000040FEE70000C5
:100A4000034900200969C90700D001207047000050
:100A5000001C004070B50446184D17482860A07966
:100A6000002802D02068410107E015487D21C90017
:100A70000068FFF73DFB21684143124802680160AE
:100A8000816808229143A279D207120F1143816035
:100A90008168022291432279D207920F114381602B
:100AA0008168042291436279D207520F1143816019
:100AB0000020286070BD000051E5CC1A001D0040E8
:100AC000F0000020001C00407047000030B5C40654
:100AD000E40E0123A340002A10D08408094AA40090
:100AE000A21814688007C00EFF2585408907090EEB
:100AF000AC43814021431160034801E0024880304B
:100B0000036030BD00E400E000E100E07047000059
:100B10000121074A89070A60064A136880079B0873
:100B20009B00800F034313600020086070470000A3
:100B30009669AA55400000407047000003480168CC
:100B4000491C01604168491C41607047F400002065
:100B5000084A03680021536191610379002B00D09A
:100B6000042143790220002B01D0014300E081439E
:100B70001161704700E000E010B50020FFF7C8FFEA
:100B800010BD026906239A430B789B075B0F1A433B
:100B90000261026908239A434B78DB071B0F1A4353
:100BA0000261026930239A438B789B079B0E1A439C
:100BB00002610269C0239A43CB789B071B0E1A433C
:100BC0000261C2680979120A1202491EC9B20A43B7
:100BD000C26081698022914381617047016949083F
:100BE00049000161704701690122114301617047A9
:100BF000026903231B0389079A43890C0A43026194
:100C00007047826903231B0389079A43890C0A43AF
:100C100082617047026903239B0389079A43090C89
:100C20000A4302617047826903239B0389079A4341
:100C3000090C0A438261704782690B78520852009E
:100C4000DB07DB0F1A438261826902239A434B78E8
:100C5000DB079B0F1A438261826904239A438B78D6
:100C6000DB075B0F1A438261826908239A43CB78C2
:100C7000DB071B0F1A438261826930239A430B7989
:100C80009B079B0E1A438261826940239A434B79EA
:100C9000DB075B0E1A438261826989798023C90769
:100CA0009A43090E0A4382617047036901221204C4
:100CB0009343036143681B0C1B040B4343600169AE
:100CC000114301617047826B120C12040A43826364
:100CD0007047C26B120C12040A43C2637047426C25
:100CE000120C12040A4342647047000010B5044C11
:100CF000204600F089F80146204600F088F810BD33
:100D000000600040C16170470246D26900200A427B
:100D100000D001207047012A826902D08A43826193
:100D200070470A43FBE70000F8B50D460E7B3449D7
:100D3000044600200F68012E06D0022E07D0032E95
:100D400008D0042E09D013E0A868000107E0A868C5
:100D5000400104E0A868800101E0A868C001FFF735
:100D600039FA00903846FFF735FA0099FFF7E8F9AD
:100D70007F21C905884202DA0020224901E0FFF7FD
:100D800044FAFFF756FA0421FFF718FAFFF729FA99
:100D900061680722120291437207520D114361608C
:100DA000206120680121490388432978C907890CFB
:100DB0000843206020680F210902884369780907E9
:100DC000090D084320602068012109038843A978A0
:100DD000C907C90C0843206020680F210906884311
:100DE000E9780907090908432060206801210907FB
:100DF00088432979C907C90808432060F8BD000065
:100E0000F00000200000F03F2030007970472030D3
:100E1000017070474268890792089200890F0A435F
:100E2000426070471CB50A487D21C9000068FFF781
:100E30005FF9009001206946087148716846FFF724
:100E400087FE044801694908490001611CBD000092
:100E5000F000002000E000E00FB410B503A9044B3F
:100E6000044A029800F024F810BC08BC04B01847EB
:100E7000FD100000FC00002030B47446641E25788C
:100E8000641CAB4200D21D46635D5B00E31830BCBE
:100E9000184702E008C8121F08C1002AFAD170479B
:100EA0007047002001E001C1121F002AFBD17047EA
:100EB000FFB58DB00446002506E025280AD0109A1B
:100EC0000F999047641C6D1C20780028F5D12846A6
:100ED00011B0F0BD00270121484A009700E0074308
:100EE000641C23780846203B98401042F7D12078B4
:100EF0002E2817D1042007436078641C2A280CD1BF
:100F00000E98641C02C800910E900BE000990A2212
:100F1000514330394018641C009020780146303924
:100F20000929F3D920780028D1D0642808D069286D
:100F300006D075281ED0109A0F9990476D1C5BE063
:100F40000A200E99019001C90E91002802DA404250
:100F50002D2102E0390504D52B216A4611720121A9
:100F600003E0F90704D02021F7E70BAE0B910DE069
:100F70000021FAE70A200E99019001C90E91F7E7C6
:100F80000199FFF7B5F83031761E31700028F7D19E
:100F900003A8801B20300190780701D5009801E05C
:100FA000012000900199884201DD401A00E00020F4
:100FB0000027009006E002A8109AC05D0F999047A4
:100FC0006D1C7F1C0B988742F5DB04E0109A3020E3
:100FD0000F9990476D1C0099481E00900029F5DC80
:100FE00005E03078109A761C0F9990476D1C019996
:100FF000481E01900029F4DC641C65E70928010003
:1010000010B505488068002803D0401E00F054FB4E
:1010100010BD0220FAE700009C00002010B5124C21
:10102000206800F083FAFF21F531884216D900F0DC
:10103000B5F8206000F09EF801460C48827B520013
:1010400012189180817B491CC9B28173052906D091
:101050004178012902D1001D00F00AF810BD0121DC
:10106000417000218173F6E7EC0000201C01002094
:10107000024610B5002001461388491C1818921C1E
:101080000529F9DB0521FFF733F880B2054910285F
:1010900002D90878012803D10120087000F0B4FAC1
:1010A00010BD00001C01002010B50848C1680848A8
:1010B000006800F09DFB032000F042F8042000F0DF
:1010C00045FC002000F00CFA10BD00008C00002050
:1010D0008800002010B5FFF7B3FC012806D10548B1
:1010E00003490160044A0021D160016010BD000085
:1010F00051E5CC1A001D0040001C0040F8B50E4F11
:101100000646C1B200243846FFF781FE0B4D02218E
:101110003846FFF7F9FD641C002801D1AC42F6D136
:1011200002213846FFF7EEFDAC4202D10020C04359
:10113000F8BD3046F8BD000000600040E21C000031
:1011400070B50B4D06460024B44205D10120E100E4
:1011500068544919496805E00022E0002A54401902
:10116000416810468847641C032CEDDB70BD00000D
:10117000D400002010B5FFF78BF9FFF7E7F801283E
:10118000FBD0FFF7EDF80446FFF792F9204610BDBB
:101190000148007870470000000100200148006805
:1011A00070470000F40000201CB500F09FF80020FC
:1011B0006A461070012151709070507191716946AA
:1011C0001920FFF7E6F969461E20FFF7E2F96946A4
:1011D0001B20FFF7DEF969461A20FFF7DAF91CBD7C
:1011E00010B50F4CA06900F0A1F9216988420DD318
:1011F00000F028FC6078002809D0012806D10020E2
:10120000607008A0FFF728FEFFF7FAFE10BD01206E
:10121000607008A0FFF720FE00F032F910BD00005A
:1012200000010020776F726B20626567696E0D0A9E
:1012300000000000776F726B206F7665720D0A00F8
:1012400070B5124C606900F071F91149884213D3EE
:10125000FFF7A4FF6061207A0E4D01280DD00EA08B
:10126000FFF7FAFDE868401EE860207A401E207211
:10127000401EC0B200F06AFB70BD00F08FFB002082
:10128000A070686008A0FFF7E7FD70BD00010020B6
:1012900040771B009C00002074696D652033306D21
:1012A000696E0D0A0000000074696D65206F766537
:1012B000720D0A001CB57D20400100900124684693
:1012C000047144718471FFF7C5FB0648044901604D
:1012D00005498A6822438A60002101601CBD000024
:1012E00051E5CC1A001D0040001C00401CB5002038
:1012F000694600900871487188711120FFF749F91B
:1013000069460D20FFF745F969461320FFF741F9BB
:1013100069461420FFF73DF969461520FFF739F9B2
:1013200069461620FFF735F969461720FFF731F9AE
:1013300069460120FFF72DF969462A20FFF729F9B0
:101340001CBD0000012203211046FFF735FBFFF70B
:1013500013FCFFF7BDF8FFF765FD17490869012287
:101360001043086100F02AFBFFF71EFF134800F04E
:1013700097FB00F09FFAFFF79DFF00F025F9FEF7BD
:10138000C7FF0F4C00F0DEF8FFF702FF00280ED079
:101390006068022801D1FFF753FFA078012803D12C
:1013A00000F042FAFFF71CFFFFF738FE01E0FFF7FD
:1013B000EFFEFFF78FFEE5E700E000E07C00002095
:1013C0000001002010B50446FFF7E2FE02460120AE
:1013D0002949002A41D00A46543A94420AD1637AF4
:1013E000002B07D1237C002B04D1E368962B01D37B
:1013F000207410BD94420CD1627A022A09D1227C59
:10140000002A06D1E268962A03D8207400F096F9E3
:1014100010BD194A383A94420ED1627A012A0BD192
:10142000227C002A08D1E268962A05D82074134845
:10143000006800F041F910BD0F4A1C3A94420CD1EB
:10144000627A012A09D1227C002A06D1E268962A12
:1014500003D8207400F0FEF810BD8C42FCD1617AF4
:101460000129F9D1217C0029F6D1E1689629F3D828
:10147000207400F0B5F810BD60000020A40000202A
:1014800010B50548C1680548006800F0B1F90020B2
:1014900000F026F810BD00008C000020880000201D
:1014A00010B50E4904464868022801D001224A605E
:1014B000012000F015F8002C08D0012C08D0022CD7
:1014C00008D0032C01D100F069FA10BD002002E021
:1014D000012000E00220FFF733FE10BD00010020D4
:1014E00010B501460120FFF751FA10BD10B51E20BE
:1014F000FFF790F8012800D0002010BD10B51B2088
:10150000FFF788F8012800D0002010BD10B51A2080
:10151000FFF780F8012800D0002010BD10B5192079
:10152000FFF778F8012800D0002010BD01460448DC
:1015300002680068401A8A4200D2401E70470000CC
:10154000F400002010B5064C6068FFF7EFFF142888
:1015500005D9FFF723FE6060002000F08BFA10BD74
:1015600000000020012110B541401120FFF70EFAC4
:1015700010BD012110B541400D20FFF707FA10BD45
:10158000012110B541401320FFF700FA10BD0121E1
:1015900010B541401420FFF7F9F910BD012110B535
:1015A00041401720FFF7F2F910BD012110B541406D
:1015B0001620FFF7EBF910BD012110B541401520B1
:1015C000FFF7E4F910BD000010B5FFF76DFD03480B
:1015D000012181600521C16010BD00009C00002038
:1015E00010B508490878002806D0002008700028A7
:1015F00004D0FFF705FD10BD0120F7E700F08AF8E1
:1016000010BD00000001002010B5104881780029AD
:1016100003D101218170FFF747FD0D4C6069FFF791
:1016200085FFFF212D3188420CD9FFF7B7FD60619E
:101630006078002807D000206070002800D00120CA
:10164000FFF790FF10BD0120F6E700001C0100200D
:101650009C00002070B500F0F5F90C4C0C4D606852
:1016600000280AD0012807D10AA0FFF7F5FB0020C7
:10167000A870606000F004F970BD0AA0FFF7ECFBF1
:101680000120A8700B492961606070BD9C0000209A
:101690000001002073746F7020696E74657276614A
:1016A0006C000000626567696E20696E7465727611
:1016B000616C0A00E093040070B5044600F0CAF9BA
:1016C00011491248124D002C0DD0012C13D0022CC0
:1016D00008D18968006800F08BF80020A86002201B
:1016E000FFF7DEFE70BD0968006800F081F8012098
:1016F000A8600020F4E74968006800F079F802204B
:10170000A8600120ECE700008C0000208800002089
:101710009C00002010B506490020C86048600549BB
:10172000887010210448FEF700FDFFF7BDFC10BDD6
:101730009C000020000100201C010020F8B5204D75
:101740006868002802D0022804D005E00020FFF7D6
:10175000B3FF01E0FFF754FC02206860FFF71EFDB5
:1017600068610120FFF7BCFE164C0026E0680127E7
:101770000300FFF781FB0605080E1216041BE66046
:101780000020E76002E00220E060012000F0DEF8C7
:101790000CE00320E0600220F8E70420E060032072
:1017A000F4E7042000F0D2F86F60E660E1680648D4
:1017B0002972414305A0E960FFF74EFBF8BD000028
:1017C000000100209C00002040771B006F7A6F6EA4
:1017D000655F6D6573736167652E6F7A6F6E655FA8
:1017E000776F726B5F74696D6525640D0A00000088
:1017F00070B50B4C05460E462046FFF7EFF900F09A
:1018000059F8B1B22046FFF75EFA0648008881B267
:101810002046FFF75EFAA9B22046FFF760FA70BDD6
:10182000002000408800002010B50D4C2069FFF713
:101830007DFE7D21C900884210D9FFF7AFFC2061F1
:101840002078032802D200F00DF804E00320FFF70F
:1018500077FC002020702078401C207010BD000014
:101860009C00002010B505488068002804D0401E68
:10187000C0B2FFF765FC10BD0220F9E79C00002014
:1018800010B5FFF7EFFF0120FFF72AFEFFF7B8FBC7
:1018900010BD1CB500206A46107050700221917076
:1018A000D070107101215171907169461220FEF7BC
:1018B00070FE1CBD7FB500246846047244728472B9
:1018C0000321C1721F4E012502A930460395FFF77F
:1018D00058F96846047045708470C470047144718E
:1018E000857169463046FFF7A7F900213046FFF7BA
:1018F0007FF902213046FFF78DF902213046FFF7CC
:1019000080F901213046FFF78EF900213046FFF7BC
:10191000CCF90D48008881B23046FFF7D4F90A4C63
:10192000241F208881B23046FFF7D3F9208881B286
:101930003046FFF7D4F9FFF7ACFF3046FFF753F915
:101940007FBD0000002000408C00002070B50546DF
:10195000042809D0104E0024AC4212DC0120E10022
:1019600070548919496812E00020FFF7FBFD002040
:10197000FFF7FFFD0020FFF703FE0020FFF707FE43
:1019800070BD0022E000325480194168104688473B
:10199000641C042CE0DB70BDB400002010B5FFF720
:1019A00083FB044900204860C86008700249C86091
:1019B00010BD0000000100209C00002070B586B022
:1019C000002468464470012505718570C4708471D7
:1019D0004471047069462520FEF7DBFD68464570BA
:1019E00005718570C4708471447104706946242047
:1019F000FEF7CFFDE1204002049068460575C472F1
:101A000004730472447284720D4C02A92046FFF7DD
:101A10008BF90122160431462046FFF77CF900219C
:101A20002046FFF7F7F9012211461720FFF74EF87D
:101A300020682843206020683043206006B070BDD5
:101A40000060004010B5FFF7A9FB0149886110BD97
:101A50000001002010B5064CA078012806D160785E
:101A6000012803D1FFF7EEFF0020607010BD0000D9
:101A70000001002070B5094D287800280CD0002402
:101A800006E001681C206043081800F02FF8641C71
:101A9000A8684168A142F4DC70BD0000000000208D
:101AA000F8B5114FB86001203870002417E01C23EE
:101AB00025465D432B46026800210933D154006856
:101AC0002E1D80598047B968321D0B6898540868EC
:101AD00080598047B96811350968641C4855B86851
:101AE0004168A142E3DCF8BD0000002010B50446C7
:101AF000C068401CE060606880477D226169D20058
:101B0000914201D2491C6161217E814202D00021B3
:101B1000616103E06169002900D060742076617C16
:101B2000204600F001F810BD70B50D460446017A5C
:101B30000F4800268068A94211D0002D07D0E6602A
:101B400026740121617282682046904705E00221D7
:101B50006172826820469047E660257270BD31460A
:101B60006672002DFAD082682046904770BD000052
:101B7000000000207377697463686B65790000006A
:101B8000696E74657276616C6B65790074696D65F8
:101B9000726B65790000000067656172736B65792F
:101BA00000000000C41B0000000000200001000035
:101BB000920E0000C41C0000000100203004000050
:101BC000A20E000000000000000000000000000065
:101BD0008C1B00001D15000000000000000000002C
:101BE000000000000000000000000000981B000042
:101BF000ED140000000000000000000000000000E4
:101C00000000000000000000801B0000FD14000028
:101C100000000000000000000000000000000000C4
:101C200000000000741B00000D1500000000000003
:101C300000000000000000000000000000000000A4
:101C40000C00002004000000C513000080BB000051
:101C500000000000E02E0000C05D00007FBB00001F
:101C60000001000000000000010000000000000072
:101C700000000000000000000000000065150000EA
:101C80000000000073150000000000008115000036
:101C9000000000008F15000000000000B9150000D2
:101CA00000000000AB150000000000009D150000C2
:101CB00000000000006CDC020000000000000000DA
:041CC0000000000020
:04000005000000C136
:00000001FF
